 fontdump

 Timestamp is 4a8b38ed (Wed Aug 19 07:27:41 2009)

 Preferred load address is 00400000

 Start         Length     Name                   Class
 0001:00000000 0000a9b4H .text                   CODE
 0002:00000000 00000124H .idata$5                DATA
 0002:00000124 00000004H .CRT$XCA                DATA
 0002:00000128 00000004H .CRT$XCZ                DATA
 0002:0000012c 00000004H .CRT$XIA                DATA
 0002:00000130 00000014H .CRT$XIC                DATA
 0002:00000144 00000004H .CRT$XIY                DATA
 0002:00000148 00000004H .CRT$XIZ                DATA
 0002:0000014c 00000004H .CRT$XPA                DATA
 0002:00000150 00000004H .CRT$XPX                DATA
 0002:00000154 00000004H .CRT$XPXA               DATA
 0002:00000158 00000004H .CRT$XPZ                DATA
 0002:0000015c 00000004H .CRT$XTA                DATA
 0002:00000160 00000004H .CRT$XTZ                DATA
 0002:00000170 00001250H .rdata                  DATA
 0002:000013c0 0000004eH .rdata$debug            DATA
 0002:00001410 0000000cH .rdata$sxdata           DATA
 0002:0000141c 00000004H .rtc$IAA                DATA
 0002:00001420 00000004H .rtc$IZZ                DATA
 0002:00001424 00000004H .rtc$TAA                DATA
 0002:00001428 00000004H .rtc$TZZ                DATA
 0002:00001430 00000474H .xdata$x                DATA
 0002:000018a4 00000014H .idata$2                DATA
 0002:000018b8 00000014H .idata$3                DATA
 0002:000018cc 00000124H .idata$4                DATA
 0002:000019f0 00000518H .idata$6                DATA
 0002:00001f08 00000000H .edata                  DATA
 0003:00000000 0000113aH .data                   DATA
 0003:00001140 00001be4H .bss                    DATA

  Address         Publics by Value              Rva+Base       Lib:Object

 0000:00000000       __except_list              00000000     <absolute>
 0000:00000003       ___safe_se_handler_count   00000003     <absolute>
 0000:00000000       ___ImageBase               00400000     <linker-defined>
 0001:00000057       _main                      00401057 f   fontdump.obj
 0001:000001e3       @__security_check_cookie@4 004011e3 f   LIBCMT:secchk.obj
 0001:000001f2       ___iob_func                004011f2 f   LIBCMT:_file.obj
 0001:000001f8       ___initstdio               004011f8 f   LIBCMT:_file.obj
 0001:000002a9       ___endstdio                004012a9 f   LIBCMT:_file.obj
 0001:000002c9       __lock_file                004012c9 f   LIBCMT:_file.obj
 0001:00000305       __lock_file2               00401305 f   LIBCMT:_file.obj
 0001:00000333       __unlock_file              00401333 f   LIBCMT:_file.obj
 0001:00000369       __unlock_file2             00401369 f   LIBCMT:_file.obj
 0001:00000393       _fgetc                     00401393 f   LIBCMT:fgetc.obj
 0001:000004ca       __fsopen                   004014ca f   LIBCMT:fopen.obj
 0001:0000058e       _fopen                     0040158e f   LIBCMT:fopen.obj
 0001:000005a1       _fprintf                   004015a1 f   LIBCMT:fprintf.obj
 0001:000006f0       _strrchr                   004016f0 f   LIBCMT:strrchr.obj
 0001:0000071d       __fclose_nolock            0040171d f   LIBCMT:fclose.obj
 0001:0000078f       _fclose                    0040178f f   LIBCMT:fclose.obj
 0001:00000a26       _mainCRTStartup            00401a26 f   LIBCMT:crt0.obj
 0001:00000a30       ___report_gsfailure        00401a30 f   LIBCMT:gs_report.obj
 0001:00000b34       __ioinit                   00401b34 f   LIBCMT:ioinit.obj
 0001:00000d74       __malloc_crt               00401d74 f   LIBCMT:crtheap.obj
 0001:00000db4       __calloc_crt               00401db4 f   LIBCMT:crtheap.obj
 0001:00000dfc       __realloc_crt              00401dfc f   LIBCMT:crtheap.obj
 0001:00000e47       _free                      00401e47 f   LIBCMT:free.obj
 0001:00000ed5       __fcloseall                00401ed5 f   LIBCMT:closeall.obj
 0001:00000f74       __amsg_exit                00401f74 f   LIBCMT:crt0dat.obj
 0001:00000f98       ___crtCorExitProcess       00401f98 f   LIBCMT:crt0dat.obj
 0001:00000fbe       ___crtExitProcess          00401fbe f   LIBCMT:crt0dat.obj
 0001:00000fd3       __lockexit                 00401fd3 f   LIBCMT:crt0dat.obj
 0001:00000fdc       __unlockexit               00401fdc f   LIBCMT:crt0dat.obj
 0001:00000ffd       __initterm_e               00401ffd f   LIBCMT:crt0dat.obj
 0001:0000101d       __get_osplatform           0040201d f   LIBCMT:crt0dat.obj
 0001:00001054       __get_winmajor             00402054 f   LIBCMT:crt0dat.obj
 0001:00001090       __cinit                    00402090 f   LIBCMT:crt0dat.obj
 0001:00001204       _exit                      00402204 f   LIBCMT:crt0dat.obj
 0001:00001215       __exit                     00402215 f   LIBCMT:crt0dat.obj
 0001:00001226       __cexit                    00402226 f   LIBCMT:crt0dat.obj
 0001:00001235       __c_exit                   00402235 f   LIBCMT:crt0dat.obj
 0001:00001244       __init_pointers            00402244 f   LIBCMT:crt0dat.obj
 0001:00001290       __flush                    00402290 f   LIBCMT:fflush.obj
 0001:000012f2       __fflush_nolock            004022f2 f   LIBCMT:fflush.obj
 0001:0000140e       __flushall                 0040240e f   LIBCMT:fflush.obj
 0001:00001417       __mtinitlocks              00402417 f   LIBCMT:mlock.obj
 0001:00001460       __mtdeletelocks            00402460 f   LIBCMT:mlock.obj
 0001:000014b5       __unlock                   004024b5 f   LIBCMT:mlock.obj
 0001:000014ca       __mtinitlocknum            004024ca f   LIBCMT:mlock.obj
 0001:0000158d       __lock                     0040258d f   LIBCMT:mlock.obj
 0001:000015be       __filbuf                   004025be f   LIBCMT:_filbuf.obj
 0001:000016de       __fileno                   004026de f   LIBCMT:fileno.obj
 0001:0000170b       __initp_misc_invarg        0040270b f   LIBCMT:invarg.obj
 0001:00001715       __invoke_watson            00402715 f   LIBCMT:invarg.obj
 0001:00001811       __invalid_parameter        00402811 f   LIBCMT:invarg.obj
 0001:00001835       __get_errno_from_oserr     00402835 f   LIBCMT:dosmap.obj
 0001:00001870       __errno                    00402870 f   LIBCMT:dosmap.obj
 0001:00001883       ___doserrno                00402883 f   LIBCMT:dosmap.obj
 0001:00001896       __dosmaperr                00402896 f   LIBCMT:dosmap.obj
 0001:000018b4       __SEH_prolog4              004028b4 f   LIBCMT:sehprolg4.obj
 0001:000018f9       __SEH_epilog4              004028f9 f   LIBCMT:sehprolg4.obj
 0001:00001910       __except_handler4          00402910 f   LIBCMT:chandler4.obj
 0001:00001aa6       __openfile                 00402aa6 f   LIBCMT:_open.obj
 0001:00001d46       __getstream                00402d46 f   LIBCMT:stream.obj
 0001:00001e78       __local_unwind4            00402e78 f   LIBCMT:exsup4.obj
 0001:00001f4e       __seh_longjmp_unwind4@4    00402f4e f   LIBCMT:exsup4.obj
 0001:00001f6a       @_EH4_CallFilterFunc@8     00402f6a f   LIBCMT:exsup4.obj
 0001:00001f81       @_EH4_TransferToHandler@8  00402f81 f   LIBCMT:exsup4.obj
 0001:00001f9a       @_EH4_GlobalUnwind@4       00402f9a f   LIBCMT:exsup4.obj
 0001:00001fb4       @_EH4_LocalUnwind@16       00402fb4 f   LIBCMT:exsup4.obj
 0001:00001fcb       __stbuf                    00402fcb f   LIBCMT:_sftbuf.obj
 0001:00002061       __ftbuf                    00403061 f   LIBCMT:_sftbuf.obj
 0001:00002090       ??0_LocaleUpdate@@QAE@PAUlocaleinfo_struct@@@Z 00403090 f i LIBCMT:output.obj
 0001:000021b3       __output_l                 004031b3 f   LIBCMT:output.obj
 0001:00002b47       __close_nolock             00403b47 f   LIBCMT:close.obj
 0001:00002bdb       __close                    00403bdb f   LIBCMT:close.obj
 0001:00002ca8       __freebuf                  00403ca8 f   LIBCMT:_freebuf.obj
 0001:00002cd4       ?__CxxUnhandledExceptionFilter@@YGJPAU_EXCEPTION_POINTERS@@@Z 00403cd4 f   LIBCMT:unhandld.obj
 0001:00002d11       ___CxxSetUnhandledExceptionFilter 00403d11 f   LIBCMT:unhandld.obj
 0001:00002d1f       __NMSG_WRITE               00403d1f f   LIBCMT:crt0msg.obj
 0001:00002ebf       __FF_MSGBANNER             00403ebf f   LIBCMT:crt0msg.obj
 0001:00002ef8       __initp_misc_winxfltr      00403ef8 f   LIBCMT:winxfltr.obj
 0001:00002ef9       __XcptFilter               00403ef9 f   LIBCMT:winxfltr.obj
 0001:00003057       __setenvp                  00404057 f   LIBCMT:stdenvp.obj
 0001:000032ca       __setargv                  004042ca f   LIBCMT:stdargv.obj
 0001:00003383       ___crtGetEnvironmentStringsA 00404383 f   LIBCMT:a_env.obj
 0001:000034b8       __RTC_Initialize           004044b8 f   LIBCMT:initsect.obj
 0001:000034dc       __RTC_Terminate            004044dc f   LIBCMT:initsect.obj
 0001:0000356c       __encode_pointer           0040456c f   LIBCMT:tidtable.obj
 0001:000035da       __encoded_null             004045da f   LIBCMT:tidtable.obj
 0001:000035e3       __decode_pointer           004045e3 f   LIBCMT:tidtable.obj
 0001:00003651       ___crtTlsAlloc@4           00404651 f   LIBCMT:tidtable.obj
 0001:0000365a       ___set_flsgetvalue         0040465a f   LIBCMT:tidtable.obj
 0001:0000368c       __mtterm                   0040468c f   LIBCMT:tidtable.obj
 0001:000036c9       __initptd                  004046c9 f   LIBCMT:tidtable.obj
 0001:00003788       __getptd_noexit            00404788 f   LIBCMT:tidtable.obj
 0001:000037ff       __getptd                   004047ff f   LIBCMT:tidtable.obj
 0001:00003817       __freefls@4                00404817 f   LIBCMT:tidtable.obj
 0001:00003938       __mtinit                   00404938 f   LIBCMT:tidtable.obj
 0001:00003abc       ___heap_select             00404abc f   LIBCMT:heapinit.obj
 0001:00003b17       __heap_init                00404b17 f   LIBCMT:heapinit.obj
 0001:00003b71       ___security_init_cookie    00404b71 f   LIBCMT:gs_support.obj
 0001:00003c05       __crt_debugger_hook        00404c05 f   LIBCMT:dbghook.obj
 0001:00003c0d       __initp_misc_initcrit      00404c0d f   LIBCMT:initcrit.obj
 0001:00003c27       ___crtInitCritSecAndSpinCount 00404c27 f   LIBCMT:initcrit.obj
 0001:00003cec       _V6_HeapAlloc              00404cec f   LIBCMT:malloc.obj
 0001:00003d3b       _malloc                    00404d3b f   LIBCMT:malloc.obj
 0001:00003dfe       __calloc_impl              00404dfe f   LIBCMT:calloc.obj
 0001:00003f1c       _realloc                   00404f1c f   LIBCMT:realloc.obj
 0001:00004137       ___sbh_heap_init           00405137 f   LIBCMT:sbheap.obj
 0001:0000417f       ___sbh_find_block          0040517f f   LIBCMT:sbheap.obj
 0001:000041aa       ___sbh_free_block          004051aa f   LIBCMT:sbheap.obj
 0001:000044be       ___sbh_alloc_new_region    004054be f   LIBCMT:sbheap.obj
 0001:0000456e       ___sbh_alloc_new_group     0040556e f   LIBCMT:sbheap.obj
 0001:00004674       ___sbh_resize_block        00405674 f   LIBCMT:sbheap.obj
 0001:00004953       ___sbh_alloc_block         00405953 f   LIBCMT:sbheap.obj
 0001:00004cef       ___onexitinit              00405cef f   LIBCMT:onexit.obj
 0001:00004d1e       __onexit                   00405d1e f   LIBCMT:onexit.obj
 0001:00004d5a       _atexit                    00405d5a f   LIBCMT:onexit.obj
 0001:00004d6c       __initp_misc_cfltcvt_tab   00405d6c f   LIBCMT:cmiscdat.obj
 0001:00004d90       __ValidateImageBase        00405d90 f   LIBCMT:pesect.obj
 0001:00004dc0       __FindPESection            00405dc0 f   LIBCMT:pesect.obj
 0001:00004e10       __IsNonwritableInCurrentImage 00405e10 f   LIBCMT:pesect.obj
 0001:00004ecb       ?terminate@@YAXXZ          00405ecb f   LIBCMT:hooks.obj
 0001:00004f04       __initp_eh_hooks           00405f04 f   LIBCMT:hooks.obj
 0001:00004f15       __initp_misc_winsig        00405f15 f   LIBCMT:winsig.obj
 0001:00004f62       ___get_sigabrt             00405f62 f   LIBCMT:winsig.obj
 0001:00004f6f       _raise                     00405f6f f   LIBCMT:winsig.obj
 0001:0000511f       __initp_misc_rand_s        0040611f f   LIBCMT:rand_s.obj
 0001:00005129       __initp_misc_purevirt      00406129 f   LIBCMT:inithelp.obj
 0001:00005133       __initp_heap_handler       00406133 f   LIBCMT:handler.obj
 0001:0000513d       __callnewh                 0040613d f   LIBCMT:handler.obj
 0001:0000515f       __write_nolock             0040615f f   LIBCMT:write.obj
 0001:00005725       __write                    00406725 f   LIBCMT:write.obj
 0001:00005801       __commit                   00406801 f   LIBCMT:commit.obj
 0001:000058e2       __read_nolock              004068e2 f   LIBCMT:read.obj
 0001:00005ea3       __read                     00406ea3 f   LIBCMT:read.obj
 0001:00005fa0       __getbuf                   00406fa0 f   LIBCMT:_getbuf.obj
 0001:00005ff0       _memset                    00406ff0 f   LIBCMT:memset.obj
 0001:000067c3       __sopen_helper             004077c3 f   LIBCMT:open.obj
 0001:0000688f       __sopen_s                  0040788f f   LIBCMT:open.obj
 0001:000068ad       __mbsicmp_l                004078ad f   LIBCMT:mbsicmp.obj
 0001:00006ac7       __mbsicmp                  00407ac7 f   LIBCMT:mbsicmp.obj
 0001:00006ada       __mbsnbcmp_l               00407ada f   LIBCMT:mbsnbcmp.obj
 0001:00006c43       __mbsnbcmp                 00407c43 f   LIBCMT:mbsnbcmp.obj
 0001:00006c5c       __global_unwind2           00407c5c f   LIBCMT:exsup.obj
 0001:00006cc1       __local_unwind2            00407cc1 f   LIBCMT:exsup.obj
 0001:00006d45       __abnormal_termination     00407d45 f   LIBCMT:exsup.obj
 0001:00006d68       __NLG_Notify1              00407d68 f   LIBCMT:exsup.obj
 0001:00006d71       __NLG_Notify               00407d71 f   LIBCMT:exsup.obj
 0001:00006d88       __NLG_Dispatch2            00407d88     LIBCMT:exsup.obj
 0001:00006d88       __NLG_Dispatch             00407d88     LIBCMT:exsup.obj
 0001:00006d90       __NLG_Call                 00407d90 f   LIBCMT:exsup.obj
 0001:00006d92       __NLG_Return2              00407d92     LIBCMT:exsup.obj
 0001:00006d93       __isatty                   00407d93 f   LIBCMT:isatty.obj
 0001:00006fff       ___updatetmbcinfo          00407fff f   LIBCMT:mbctype.obj
 0001:0000711d       __setmbcp_nolock           0040811d f   LIBCMT:mbctype.obj
 0001:000072f6       __setmbcp                  004082f6 f   LIBCMT:mbctype.obj
 0001:00007490       ___initmbctable            00408490 f   LIBCMT:mbctype.obj
 0001:000074ae       ___freetlocinfo            004084ae f   LIBCMT:setlocal.obj
 0001:000075ee       ___addlocaleref            004085ee f   LIBCMT:setlocal.obj
 0001:00007674       ___removelocaleref         00408674 f   LIBCMT:setlocal.obj
 0001:0000773e       ___updatetlocinfo          0040873e f   LIBCMT:setlocal.obj
 0001:000077b4       __flsbuf                   004087b4 f   LIBCMT:_flsbuf.obj
 0001:00007914       __get_printf_count_output  00408914 f   LIBCMT:printf.obj
 0001:00007930       _strlen                    00408930 f   LIBCMT:strlen.obj
 0001:000079bb       __wctomb_s_l               004089bb f   LIBCMT:wctomb.obj
 0001:00007b1a       _wctomb_s                  00408b1a f   LIBCMT:wctomb.obj
 0001:00007b35       __isleadbyte_l             00408b35 f i LIBCMT:_wctype.obj
 0001:00007b6b       _isleadbyte                00408b6b f i LIBCMT:_wctype.obj
 0001:00007b80       __aulldvrm                 00408b80 f   LIBCMT:ulldvrm.obj
 0001:00007c15       __set_osfhnd               00408c15 f   LIBCMT:osfinfo.obj
 0001:00007c92       __free_osfhnd              00408c92 f   LIBCMT:osfinfo.obj
 0001:00007d13       __get_osfhandle            00408d13 f   LIBCMT:osfinfo.obj
 0001:00007d84       ___lock_fhandle            00408d84 f   LIBCMT:osfinfo.obj
 0001:00007e24       __unlock_fhandle           00408e24 f   LIBCMT:osfinfo.obj
 0001:00007e46       __alloc_osfhnd             00408e46 f   LIBCMT:osfinfo.obj
 0001:00007fe5       ___crtMessageBoxA          00408fe5 f   LIBCMT:crtmbox.obj
 0001:000081a2       _strcat_s                  004091a2 f   LIBCMT:strcat_s.obj
 0001:00008213       _strncpy_s                 00409213 f   LIBCMT:strncpy_s.obj
 0001:000082c6       _strcpy_s                  004092c6 f   LIBCMT:strcpy_s.obj
 0001:0000832b       __set_error_mode           0040932b f   LIBCMT:errmode.obj
 0001:000083c2       __ismbblead                004093c2 f   LIBCMT:ismbbyte.obj
 0001:000083e0       _memcpy                    004093e0 f   LIBCMT:memcpy.obj
 0001:00008750       _strcmp                    00409750 f   LIBCMT:strcmp.obj
 0001:000087d8       __msize                    004097d8 f   LIBCMT:msize.obj
 0001:00008880       _memmove                   00409880 f   LIBCMT:memmove.obj
 0001:00008be5       __fptrap                   00409be5 f   LIBCMT:crt0fp.obj
 0001:00008bee       _abort                     00409bee f   LIBCMT:abort.obj
 0001:00008ce1       __freea                    00409ce1 f i LIBCMT:w_loc.obj
 0001:00008cfc       __putwch_nolock            00409cfc f   LIBCMT:putwch.obj
 0001:00008dbe       __mbtowc_l                 00409dbe f   LIBCMT:mbtowc.obj
 0001:00008ed1       _mbtowc                    00409ed1 f   LIBCMT:mbtowc.obj
 0001:00008ee8       __lseeki64_nolock          00409ee8 f   LIBCMT:lseeki64.obj
 0001:00008f6b       __lseeki64                 00409f6b f   LIBCMT:lseeki64.obj
 0001:000090db       __VEC_memzero              0040a0db f   LIBCMT:p4_memset.obj
 0001:0000916a       __sse2_mathfcns_init       0040a16a f   LIBCMT:mathfcns.obj
 0001:0000917e       __chsize_nolock            0040a17e f   LIBCMT:chsize.obj
 0001:00009332       __lseek_nolock             0040a332 f   LIBCMT:lseek.obj
 0001:000093a4       __setmode_nolock           0040a3a4 f   LIBCMT:setmode.obj
 0001:00009460       __get_fmode                0040a460 f   LIBCMT:setmode.obj
 0001:00009836       ___crtLCMapStringA         0040a836 f   LIBCMT:a_map.obj
 0001:00009879       ___ascii_stricmp           0040a879 f   LIBCMT:stricmp.obj
 0001:000098ae       __stricmp_l                0040a8ae f   LIBCMT:stricmp.obj
 0001:00009981       _strncmp                   0040a981 f   LIBCMT:strncmp.obj
 0001:00009bf7       ___crtGetStringTypeA       0040abf7 f   LIBCMT:a_str.obj
 0001:00009c37       ___free_lc_time            0040ac37 f   LIBCMT:inittime.obj
 0001:00009dc7       ___free_lconv_num          0040adc7 f   LIBCMT:initnum.obj
 0001:00009e07       ___free_lconv_mon          0040ae07 f   LIBCMT:initmon.obj
 0001:00009e90       _strcspn                   0040ae90 f   LIBCMT:strcspn.obj
 0001:00009ee0       _strpbrk                   0040aee0 f   LIBCMT:strpbrk.obj
 0001:0000a14b       _strtol                    0040b14b f   LIBCMT:strtol.obj
 0001:0000a1fb       __VEC_memcpy               0040b1fb f   LIBCMT:p4_memcpy.obj
 0001:0000a2de       __isctype_l                0040b2de f   LIBCMT:isctype.obj
 0001:0000a3a0       __alloca_probe_16          0040b3a0 f   LIBCMT:alloca16.obj
 0001:0000a3b6       __alloca_probe_8           0040b3b6     LIBCMT:alloca16.obj
 0001:0000a3cc       ___initconout              0040b3cc f   LIBCMT:initcon.obj
 0001:0000a3eb       ___termcon                 0040b3eb f   LIBCMT:initcon.obj
 0001:0000a468       __get_sse2_info            0040b468 f   LIBCMT:cpu_disp.obj
 0001:0000a4c8       ___sse2_available_init     0040b4c8 f   LIBCMT:cpu_disp.obj
 0001:0000a4d5       ___ansicp                  0040b4d5 f   LIBCMT:convrtcp.obj
 0001:0000a51c       ___convertcp               0040b51c f   LIBCMT:convrtcp.obj
 0001:0000a6ce       __tolower_l                0040b6ce f   LIBCMT:tolower.obj
 0001:0000a7e5       _atol                      0040b7e5 f   LIBCMT:atox.obj
 0001:0000a800       __chkstk                   0040b800 f   LIBCMT:chkstk.obj
 0001:0000a800       __alloca_probe             0040b800     LIBCMT:chkstk.obj
 0001:0000a830       ___ascii_strnicmp          0040b830 f   LIBCMT:_strnicm.obj
 0001:0000a8a0       __allmul                   0040b8a0 f   LIBCMT:llmul.obj
 0001:0000a8f0       _strchr                    0040b8f0 f   LIBCMT:strchr.obj
 0001:0000a8f6       ___from_strstr_to_strchr   0040b8f6     LIBCMT:strchr.obj
 0001:0000a9ae       _RtlUnwind@16              0040b9ae f   kernel32:KERNEL32.dll
 0002:00000000       __imp__EnterCriticalSection@4 0040c000     kernel32:KERNEL32.dll
 0002:00000004       __imp__LeaveCriticalSection@4 0040c004     kernel32:KERNEL32.dll
 0002:00000008       __imp__GetCommandLineA@0   0040c008     kernel32:KERNEL32.dll
 0002:0000000c       __imp__HeapFree@12         0040c00c     kernel32:KERNEL32.dll
 0002:00000010       __imp__GetVersionExA@4     0040c010     kernel32:KERNEL32.dll
 0002:00000014       __imp__HeapAlloc@12        0040c014     kernel32:KERNEL32.dll
 0002:00000018       __imp__GetProcessHeap@0    0040c018     kernel32:KERNEL32.dll
 0002:0000001c       __imp__TerminateProcess@8  0040c01c     kernel32:KERNEL32.dll
 0002:00000020       __imp__GetCurrentProcess@0 0040c020     kernel32:KERNEL32.dll
 0002:00000024       __imp__UnhandledExceptionFilter@4 0040c024     kernel32:KERNEL32.dll
 0002:00000028       __imp__SetUnhandledExceptionFilter@4 0040c028     kernel32:KERNEL32.dll
 0002:0000002c       __imp__IsDebuggerPresent@0 0040c02c     kernel32:KERNEL32.dll
 0002:00000030       __imp__SetHandleCount@4    0040c030     kernel32:KERNEL32.dll
 0002:00000034       __imp__GetStdHandle@4      0040c034     kernel32:KERNEL32.dll
 0002:00000038       __imp__GetFileType@4       0040c038     kernel32:KERNEL32.dll
 0002:0000003c       __imp__GetStartupInfoA@4   0040c03c     kernel32:KERNEL32.dll
 0002:00000040       __imp__DeleteCriticalSection@4 0040c040     kernel32:KERNEL32.dll
 0002:00000044       __imp__Sleep@4             0040c044     kernel32:KERNEL32.dll
 0002:00000048       __imp__GetLastError@0      0040c048     kernel32:KERNEL32.dll
 0002:0000004c       __imp__GetProcAddress@8    0040c04c     kernel32:KERNEL32.dll
 0002:00000050       __imp__GetModuleHandleA@4  0040c050     kernel32:KERNEL32.dll
 0002:00000054       __imp__ExitProcess@4       0040c054     kernel32:KERNEL32.dll
 0002:00000058       __imp__RtlUnwind@16        0040c058     kernel32:KERNEL32.dll
 0002:0000005c       __imp__CloseHandle@4       0040c05c     kernel32:KERNEL32.dll
 0002:00000060       __imp__WriteFile@20        0040c060     kernel32:KERNEL32.dll
 0002:00000064       __imp__GetModuleFileNameA@12 0040c064     kernel32:KERNEL32.dll
 0002:00000068       __imp__FreeEnvironmentStringsA@4 0040c068     kernel32:KERNEL32.dll
 0002:0000006c       __imp__GetEnvironmentStrings@0 0040c06c     kernel32:KERNEL32.dll
 0002:00000070       __imp__FreeEnvironmentStringsW@4 0040c070     kernel32:KERNEL32.dll
 0002:00000074       __imp__WideCharToMultiByte@32 0040c074     kernel32:KERNEL32.dll
 0002:00000078       __imp__GetEnvironmentStringsW@0 0040c078     kernel32:KERNEL32.dll
 0002:0000007c       __imp__TlsGetValue@4       0040c07c     kernel32:KERNEL32.dll
 0002:00000080       __imp__TlsAlloc@0          0040c080     kernel32:KERNEL32.dll
 0002:00000084       __imp__TlsSetValue@8       0040c084     kernel32:KERNEL32.dll
 0002:00000088       __imp__TlsFree@4           0040c088     kernel32:KERNEL32.dll
 0002:0000008c       __imp__InterlockedIncrement@4 0040c08c     kernel32:KERNEL32.dll
 0002:00000090       __imp__SetLastError@4      0040c090     kernel32:KERNEL32.dll
 0002:00000094       __imp__GetCurrentThreadId@0 0040c094     kernel32:KERNEL32.dll
 0002:00000098       __imp__InterlockedDecrement@4 0040c098     kernel32:KERNEL32.dll
 0002:0000009c       __imp__HeapDestroy@4       0040c09c     kernel32:KERNEL32.dll
 0002:000000a0       __imp__HeapCreate@12       0040c0a0     kernel32:KERNEL32.dll
 0002:000000a4       __imp__VirtualFree@12      0040c0a4     kernel32:KERNEL32.dll
 0002:000000a8       __imp__QueryPerformanceCounter@4 0040c0a8     kernel32:KERNEL32.dll
 0002:000000ac       __imp__GetTickCount@0      0040c0ac     kernel32:KERNEL32.dll
 0002:000000b0       __imp__GetCurrentProcessId@0 0040c0b0     kernel32:KERNEL32.dll
 0002:000000b4       __imp__GetSystemTimeAsFileTime@4 0040c0b4     kernel32:KERNEL32.dll
 0002:000000b8       __imp__InitializeCriticalSection@4 0040c0b8     kernel32:KERNEL32.dll
 0002:000000bc       __imp__HeapReAlloc@16      0040c0bc     kernel32:KERNEL32.dll
 0002:000000c0       __imp__VirtualAlloc@16     0040c0c0     kernel32:KERNEL32.dll
 0002:000000c4       __imp__LoadLibraryA@4      0040c0c4     kernel32:KERNEL32.dll
 0002:000000c8       __imp__GetConsoleCP@0      0040c0c8     kernel32:KERNEL32.dll
 0002:000000cc       __imp__GetConsoleMode@8    0040c0cc     kernel32:KERNEL32.dll
 0002:000000d0       __imp__FlushFileBuffers@4  0040c0d0     kernel32:KERNEL32.dll
 0002:000000d4       __imp__MultiByteToWideChar@24 0040c0d4     kernel32:KERNEL32.dll
 0002:000000d8       __imp__ReadFile@20         0040c0d8     kernel32:KERNEL32.dll
 0002:000000dc       __imp__CreateFileA@28      0040c0dc     kernel32:KERNEL32.dll
 0002:000000e0       __imp__GetCPInfo@8         0040c0e0     kernel32:KERNEL32.dll
 0002:000000e4       __imp__GetACP@0            0040c0e4     kernel32:KERNEL32.dll
 0002:000000e8       __imp__GetOEMCP@0          0040c0e8     kernel32:KERNEL32.dll
 0002:000000ec       __imp__IsValidCodePage@4   0040c0ec     kernel32:KERNEL32.dll
 0002:000000f0       __imp__SetStdHandle@8      0040c0f0     kernel32:KERNEL32.dll
 0002:000000f4       __imp__HeapSize@12         0040c0f4     kernel32:KERNEL32.dll
 0002:000000f8       __imp__GetLocaleInfoA@16   0040c0f8     kernel32:KERNEL32.dll
 0002:000000fc       __imp__WriteConsoleA@20    0040c0fc     kernel32:KERNEL32.dll
 0002:00000100       __imp__GetConsoleOutputCP@0 0040c100     kernel32:KERNEL32.dll
 0002:00000104       __imp__WriteConsoleW@20    0040c104     kernel32:KERNEL32.dll
 0002:00000108       __imp__SetFilePointer@16   0040c108     kernel32:KERNEL32.dll
 0002:0000010c       __imp__SetEndOfFile@4      0040c10c     kernel32:KERNEL32.dll
 0002:00000110       __imp__LCMapStringA@24     0040c110     kernel32:KERNEL32.dll
 0002:00000114       __imp__LCMapStringW@24     0040c114     kernel32:KERNEL32.dll
 0002:00000118       __imp__GetStringTypeA@20   0040c118     kernel32:KERNEL32.dll
 0002:0000011c       __imp__GetStringTypeW@16   0040c11c     kernel32:KERNEL32.dll
 0002:00000120       \177KERNEL32_NULL_THUNK_DATA 0040c120     kernel32:KERNEL32.dll
 0002:00000124       ___xc_a                    0040c124     LIBCMT:crt0init.obj
 0002:00000128       ___xc_z                    0040c128     LIBCMT:crt0init.obj
 0002:0000012c       ___xi_a                    0040c12c     LIBCMT:crt0init.obj
 0002:00000148       ___xi_z                    0040c148     LIBCMT:crt0init.obj
 0002:0000014c       ___xp_a                    0040c14c     LIBCMT:crt0init.obj
 0002:00000158       ___xp_z                    0040c158     LIBCMT:crt0init.obj
 0002:0000015c       ___xt_a                    0040c15c     LIBCMT:crt0init.obj
 0002:00000160       ___xt_z                    0040c160     LIBCMT:crt0init.obj
 0002:00000194       ??_C@_0P@MIGLKIOC@CorExitProcess?$AA@ 0040c194     LIBCMT:crt0dat.obj
 0002:000001a4       ??_C@_0M@MBOPBNBK@mscoree?4dll?$AA@ 0040c1a4     LIBCMT:crt0dat.obj
 0002:000001d4       ??_C@_1O@CEDCILHN@?$AA?$CI?$AAn?$AAu?$AAl?$AAl?$AA?$CJ?$AA?$AA@ 0040c1d4     LIBCMT:output.obj
 0002:000001e4       ??_C@_06OJHGLDPL@?$CInull?$CJ?$AA@ 0040c1e4     LIBCMT:output.obj
 0002:000001f0       ___lookuptable             0040c1f0     LIBCMT:output.obj
 0002:0000024c       ??_C@_0P@GGKDKEEG@runtime?5error?5?$AA@ 0040c24c     LIBCMT:crt0msg.obj
 0002:0000025c       ??_C@_02PCIJFNDE@?$AN?6?$AA@ 0040c25c     LIBCMT:crt0msg.obj
 0002:00000260       ??_C@_0O@MJNIPGOH@TLOSS?5error?$AN?6?$AA@ 0040c260     LIBCMT:crt0msg.obj
 0002:00000270       ??_C@_0N@BONNPDHF@SING?5error?$AN?6?$AA@ 0040c270     LIBCMT:crt0msg.obj
 0002:00000280       ??_C@_0P@MBDAJNE@DOMAIN?5error?$AN?6?$AA@ 0040c280     LIBCMT:crt0msg.obj
 0002:00000290       ??_C@_0JL@DFDOOABL@R6034?$AN?6An?5application?5has?5made?5a@ 0040c290     LIBCMT:crt0msg.obj
 0002:00000330       ??_C@_0PH@EPAFIJ@R6033?$AN?6?9?5Attempt?5to?5use?5MSIL?5cod@ 0040c330     LIBCMT:crt0msg.obj
 0002:00000428       ??_C@_0DD@BKEEABMM@R6032?$AN?6?9?5not?5enough?5space?5for?5lo@ 0040c428     LIBCMT:crt0msg.obj
 0002:00000460       ??_C@_0GD@OFKILIED@R6031?$AN?6?9?5Attempt?5to?5initialize?5t@ 0040c460     LIBCMT:crt0msg.obj
 0002:000004c4       ??_C@_0BP@LPMHJOKI@R6030?$AN?6?9?5CRT?5not?5initialized?$AN?6?$AA@ 0040c4c4     LIBCMT:crt0msg.obj
 0002:000004e4       ??_C@_0CF@KJDAIALP@R6028?$AN?6?9?5unable?5to?5initialize?5he@ 0040c4e4     LIBCMT:crt0msg.obj
 0002:0000050c       ??_C@_0DF@GAKBPDFP@R6027?$AN?6?9?5not?5enough?5space?5for?5lo@ 0040c50c     LIBCMT:crt0msg.obj
 0002:00000544       ??_C@_0DF@IBLNNAIG@R6026?$AN?6?9?5not?5enough?5space?5for?5st@ 0040c544     LIBCMT:crt0msg.obj
 0002:0000057c       ??_C@_0CG@IOHKGFNJ@R6025?$AN?6?9?5pure?5virtual?5function?5c@ 0040c57c     LIBCMT:crt0msg.obj
 0002:000005a4       ??_C@_0DF@JIJJFJDC@R6024?$AN?6?9?5not?5enough?5space?5for?5_o@ 0040c5a4     LIBCMT:crt0msg.obj
 0002:000005dc       ??_C@_0CJ@EGEJHFME@R6019?$AN?6?9?5unable?5to?5open?5console?5@ 0040c5dc     LIBCMT:crt0msg.obj
 0002:00000608       ??_C@_0CB@GNHNIELH@R6018?$AN?6?9?5unexpected?5heap?5error?$AN?6@ 0040c608     LIBCMT:crt0msg.obj
 0002:0000062c       ??_C@_0CN@FOLDKNG@R6017?$AN?6?9?5unexpected?5multithread?5@ 0040c62c     LIBCMT:crt0msg.obj
 0002:0000065c       ??_C@_0CM@FAHFJNHO@R6016?$AN?6?9?5not?5enough?5space?5for?5th@ 0040c65c     LIBCMT:crt0msg.obj
 0002:00000688       ??_C@_0JG@LBKMGKLD@?$AN?6This?5application?5has?5requested@ 0040c688     LIBCMT:crt0msg.obj
 0002:00000720       ??_C@_0CM@FLCNIPKK@R6009?$AN?6?9?5not?5enough?5space?5for?5en@ 0040c720     LIBCMT:crt0msg.obj
 0002:0000074c       ??_C@_0CK@KMMJOAPP@R6008?$AN?6?9?5not?5enough?5space?5for?5ar@ 0040c74c     LIBCMT:crt0msg.obj
 0002:00000778       ??_C@_0CN@LEKKICBM@R6002?$AN?6?9?5floating?5point?5support?5@ 0040c778     LIBCMT:crt0msg.obj
 0002:000007a8       ??_C@_0CF@GOGNBNAK@Microsoft?5Visual?5C?$CL?$CL?5Runtime?5Lib@ 0040c7a8     LIBCMT:crt0msg.obj
 0002:000007d0       ??_C@_02PHMGELLB@?6?6?$AA@ 0040c7d0     LIBCMT:crt0msg.obj
 0002:000007d4       ??_C@_03KHICJKCI@?4?4?4?$AA@ 0040c7d4     LIBCMT:crt0msg.obj
 0002:000007d8       ??_C@_0BH@DNAGHKFM@?$DMprogram?5name?5unknown?$DO?$AA@ 0040c7d8     LIBCMT:crt0msg.obj
 0002:000007f0       ??_C@_0BK@OFGJDLJJ@Runtime?5Error?$CB?6?6Program?3?5?$AA@ 0040c7f0     LIBCMT:crt0msg.obj
 0002:0000080c       ??_C@_07EPKMNAGK@?4mixcrt?$AA@ 0040c80c     LIBCMT:tidtable.obj
 0002:00000814       ??_C@_0O@NLDKAIKN@EncodePointer?$AA@ 0040c814     LIBCMT:tidtable.obj
 0002:00000824       ??_C@_0N@NHGLKGEC@KERNEL32?4DLL?$AA@ 0040c824     LIBCMT:tidtable.obj
 0002:00000834       ??_C@_0O@KBPMFGHI@DecodePointer?$AA@ 0040c834     LIBCMT:tidtable.obj
 0002:00000844       ??_C@_07PEJMOBNF@FlsFree?$AA@ 0040c844     LIBCMT:tidtable.obj
 0002:0000084c       ??_C@_0M@JCPCPOEF@FlsSetValue?$AA@ 0040c84c     LIBCMT:tidtable.obj
 0002:00000858       ??_C@_0M@GDNOONDI@FlsGetValue?$AA@ 0040c858     LIBCMT:tidtable.obj
 0002:00000864       ??_C@_08KNHFBNJ@FlsAlloc?$AA@ 0040c864     LIBCMT:tidtable.obj
 0002:00000870       ??_C@_0CG@PKBDLMEO@InitializeCriticalSectionAndSpin@ 0040c870     LIBCMT:initcrit.obj
 0002:00000898       ??_C@_0N@MDJJJHMB@kernel32?4dll?$AA@ 0040c898     LIBCMT:initcrit.obj
 0002:00000928       ___lookuptable_s           0040c928     LIBCMT:outputs.obj
 0002:00000984       ??_C@_0BI@DFKBFLJE@GetProcessWindowStation?$AA@ 0040c984     LIBCMT:crtmbox.obj
 0002:0000099c       ??_C@_0BK@CIDNPOGP@GetUserObjectInformationA?$AA@ 0040c99c     LIBCMT:crtmbox.obj
 0002:000009b8       ??_C@_0BD@HHGDFDBJ@GetLastActivePopup?$AA@ 0040c9b8     LIBCMT:crtmbox.obj
 0002:000009cc       ??_C@_0BA@HNOPNCHB@GetActiveWindow?$AA@ 0040c9cc     LIBCMT:crtmbox.obj
 0002:000009dc       ??_C@_0M@CHKKJDAI@MessageBoxA?$AA@ 0040c9dc     LIBCMT:crtmbox.obj
 0002:000009e8       ??_C@_0L@NDEGIDAG@USER32?4DLL?$AA@ 0040c9e8     LIBCMT:crtmbox.obj
 0002:000009f4       ??_C@_13NOLLCAOD@?$AA?$AA?$AA?$AA@ 0040c9f4     LIBCMT:a_map.obj
 0002:000009f8       ___newctype                0040c9f8     LIBCMT:ctype.obj
 0002:00000cf8       __wctype                   0040ccf8     LIBCMT:ctype.obj
 0002:00000f00       ___newclmap                0040cf00     LIBCMT:ctype.obj
 0002:00001080       ___newcumap                0040d080     LIBCMT:ctype.obj
 0002:00001200       ??_C@_08JCCMCCIL@HH?3mm?3ss?$AA@ 0040d200     LIBCMT:strftime.obj
 0002:0000120c       ??_C@_0BE@CKGJFCPC@dddd?0?5MMMM?5dd?0?5yyyy?$AA@ 0040d20c     LIBCMT:strftime.obj
 0002:00001220       ??_C@_08BPBNCDIB@MM?1dd?1yy?$AA@ 0040d220     LIBCMT:strftime.obj
 0002:0000122c       ??_C@_02CJNFDJBF@PM?$AA@   0040d22c     LIBCMT:strftime.obj
 0002:00001230       ??_C@_02DEDBPAFC@AM?$AA@   0040d230     LIBCMT:strftime.obj
 0002:00001234       ??_C@_08EDHMEBNP@December?$AA@ 0040d234     LIBCMT:strftime.obj
 0002:00001240       ??_C@_08HCHEGEOA@November?$AA@ 0040d240     LIBCMT:strftime.obj
 0002:0000124c       ??_C@_07JJNFCEND@October?$AA@ 0040d24c     LIBCMT:strftime.obj
 0002:00001254       ??_C@_09BHHEALKD@September?$AA@ 0040d254     LIBCMT:strftime.obj
 0002:00001260       ??_C@_06LBBHFDDG@August?$AA@ 0040d260     LIBCMT:strftime.obj
 0002:00001268       ??_C@_04MIEPOIFP@July?$AA@ 0040d268     LIBCMT:strftime.obj
 0002:00001270       ??_C@_04CNLMGBGM@June?$AA@ 0040d270     LIBCMT:strftime.obj
 0002:00001278       ??_C@_05DMJDNLEJ@April?$AA@ 0040d278     LIBCMT:strftime.obj
 0002:00001280       ??_C@_05HPCKOFNC@March?$AA@ 0040d280     LIBCMT:strftime.obj
 0002:00001288       ??_C@_08GNJGEPFN@February?$AA@ 0040d288     LIBCMT:strftime.obj
 0002:00001294       ??_C@_07CGJPFGJA@January?$AA@ 0040d294     LIBCMT:strftime.obj
 0002:0000129c       ??_C@_03MKABNOCG@Dec?$AA@  0040d29c     LIBCMT:strftime.obj
 0002:000012a0       ??_C@_03JPJOFNIA@Nov?$AA@  0040d2a0     LIBCMT:strftime.obj
 0002:000012a4       ??_C@_03BMAOKBAD@Oct?$AA@  0040d2a4     LIBCMT:strftime.obj
 0002:000012a8       ??_C@_03GGCAPAJC@Sep?$AA@  0040d2a8     LIBCMT:strftime.obj
 0002:000012ac       ??_C@_03IFJFEIGA@Aug?$AA@  0040d2ac     LIBCMT:strftime.obj
 0002:000012b0       ??_C@_03LBGABGKK@Jul?$AA@  0040d2b0     LIBCMT:strftime.obj
 0002:000012b4       ??_C@_03IDFGHECI@Jun?$AA@  0040d2b4     LIBCMT:strftime.obj
 0002:000012b8       ??_C@_03CNMDKL@May?$AA@    0040d2b8     LIBCMT:strftime.obj
 0002:000012bc       ??_C@_03LEOLGMJP@Apr?$AA@  0040d2bc     LIBCMT:strftime.obj
 0002:000012c0       ??_C@_03ODNJBKGA@Mar?$AA@  0040d2c0     LIBCMT:strftime.obj
 0002:000012c4       ??_C@_03HJBDCHOM@Feb?$AA@  0040d2c4     LIBCMT:strftime.obj
 0002:000012c8       ??_C@_03JIHJHPIE@Jan?$AA@  0040d2c8     LIBCMT:strftime.obj
 0002:000012cc       ??_C@_08INBOOONO@Saturday?$AA@ 0040d2cc     LIBCMT:strftime.obj
 0002:000012d8       ??_C@_06JECMNKMI@Friday?$AA@ 0040d2d8     LIBCMT:strftime.obj
 0002:000012e0       ??_C@_08HACCIKIA@Thursday?$AA@ 0040d2e0     LIBCMT:strftime.obj
 0002:000012ec       ??_C@_09DLIGFAKA@Wednesday?$AA@ 0040d2ec     LIBCMT:strftime.obj
 0002:000012f8       ??_C@_07BAAGCFCM@Tuesday?$AA@ 0040d2f8     LIBCMT:strftime.obj
 0002:00001300       ??_C@_06JLEDEDGH@Monday?$AA@ 0040d300     LIBCMT:strftime.obj
 0002:00001308       ??_C@_06OOPIFAJ@Sunday?$AA@ 0040d308     LIBCMT:strftime.obj
 0002:00001310       ??_C@_03FEFJNEK@Sat?$AA@   0040d310     LIBCMT:strftime.obj
 0002:00001314       ??_C@_03IDIOELNC@Fri?$AA@  0040d314     LIBCMT:strftime.obj
 0002:00001318       ??_C@_03IOFIKPDN@Thu?$AA@  0040d318     LIBCMT:strftime.obj
 0002:0000131c       ??_C@_03MHOMLAJA@Wed?$AA@  0040d31c     LIBCMT:strftime.obj
 0002:00001320       ??_C@_03NAGEINEP@Tue?$AA@  0040d320     LIBCMT:strftime.obj
 0002:00001324       ??_C@_03PDAGKDH@Mon?$AA@   0040d324     LIBCMT:strftime.obj
 0002:00001328       ??_C@_03KOEHGMDN@Sun?$AA@  0040d328     LIBCMT:strftime.obj
 0002:0000132c       ??_C@_07GPDNMNG@CONOUT$?$AA@ 0040d32c     LIBCMT:initcon.obj
 0002:00001334       ___dnames                  0040d334     LIBCMT:timeset.obj
 0002:0000134c       ___mnames                  0040d34c     LIBCMT:timeset.obj
 0002:00001378       __load_config_used         0040d378     LIBCMT:loadcfg.obj
 0002:00001410       ___safe_se_handler_table   0040d410     <linker-defined>
 0002:0000141c       ___rtc_iaa                 0040d41c     LIBCMT:initsect.obj
 0002:00001420       ___rtc_izz                 0040d420     LIBCMT:initsect.obj
 0002:00001424       ___rtc_taa                 0040d424     LIBCMT:initsect.obj
 0002:00001428       ___rtc_tzz                 0040d428     LIBCMT:initsect.obj
 0002:000018a4       __IMPORT_DESCRIPTOR_KERNEL32 0040d8a4     kernel32:KERNEL32.dll
 0002:000018b8       __NULL_IMPORT_DESCRIPTOR   0040d8b8     kernel32:KERNEL32.dll
 0003:00000000       __iob                      0040e000     LIBCMT:_file.obj
 0003:00000280       ___app_type                0040e280     LIBCMT:crt0.obj
 0003:00000284       ___security_cookie         0040e284     LIBCMT:gs_cookie.obj
 0003:00000288       ___security_cookie_complement 0040e288     LIBCMT:gs_cookie.obj
 0003:00000290       ___badioinfo               0040e290     LIBCMT:ioinit.obj
 0003:000002c8       __aexit_rtn                0040e2c8     LIBCMT:crt0dat.obj
 0003:00000560       ___nullstring              0040e560     LIBCMT:output.obj
 0003:00000564       ___wnullstring             0040e564     LIBCMT:output.obj
 0003:00000620       __XcptActTab               0040e620     LIBCMT:winxfltr.obj
 0003:00000698       __First_FPE_Indx           0040e698     LIBCMT:winxfltr.obj
 0003:0000069c       __Num_FPE                  0040e69c     LIBCMT:winxfltr.obj
 0003:000006a0       __XcptActTabSize           0040e6a0     LIBCMT:winxfltr.obj
 0003:000006a4       __XcptActTabCount          0040e6a4     LIBCMT:winxfltr.obj
 0003:000006a8       ___flsindex                0040e6a8     LIBCMT:tidtable.obj
 0003:000006ac       ___getvalueindex           0040e6ac     LIBCMT:tidtable.obj
 0003:000006b0       __amblksiz                 0040e6b0     LIBCMT:heapinit.obj
 0003:000006b4       __cfltcvt_tab              0040e6b4     LIBCMT:cmiscdat.obj
 0003:000006e0       __lookuptrailbytes         0040e6e0     LIBCMT:read.obj
 0003:000007e0       __NLG_Destination          0040e7e0     LIBCMT:exsup.obj
 0003:000007f0       ___initialmbcinfo          0040e7f0     LIBCMT:mbctype.obj
 0003:00000a10       __mbctype                  0040ea10     LIBCMT:mbctype.obj
 0003:00000b18       __mbcasemap                0040eb18     LIBCMT:mbctype.obj
 0003:00000c18       ___ptmbcinfo               0040ec18     LIBCMT:mbctype.obj
 0003:00000d14       ___globallocalestatus      0040ed14     LIBCMT:glstatus.obj
 0003:00000d18       ___clocalestr              0040ed18     LIBCMT:nlsdata2.obj
 0003:00000d20       ___initiallocinfo          0040ed20     LIBCMT:nlsdata2.obj
 0003:00000df8       ___ptlocinfo               0040edf8     LIBCMT:nlsdata2.obj
 0003:00000dfc       ___lc_clike                0040edfc     LIBCMT:nlsdata2.obj
 0003:00000e00       ___initiallocalestructinfo 0040ee00     LIBCMT:nlsdata2.obj
 0003:00000e10       ___abort_behavior          0040ee10     LIBCMT:abort.obj
 0003:00000e18       __pctype                   0040ee18     LIBCMT:ctype.obj
 0003:00000e1c       __pwctype                  0040ee1c     LIBCMT:ctype.obj
 0003:00000e20       ___lc_time_c               0040ee20     LIBCMT:strftime.obj
 0003:00000ed8       ___lc_time_curr            0040eed8     LIBCMT:strftime.obj
 0003:00000edc       ___lconv_static_decimal    0040eedc     LIBCMT:lconv.obj
 0003:00000ee0       ___lconv_c                 0040eee0     LIBCMT:lconv.obj
 0003:00000f10       ___lconv                   0040ef10     LIBCMT:lconv.obj
 0003:00000f14       ___mb_cur_max              0040ef14     LIBCMT:nlsdata1.obj
 0003:00000f18       ___decimal_point           0040ef18     LIBCMT:nlsdata1.obj
 0003:00000f1c       ___decimal_point_length    0040ef1c     LIBCMT:nlsdata1.obj
 0003:00000f20       __coninpfh                 0040ef20     LIBCMT:initcon.obj
 0003:00000f24       __confh                    0040ef24     LIBCMT:initcon.obj
 0003:00000f28       __timezone                 0040ef28     LIBCMT:timeset.obj
 0003:00000f2c       __daylight                 0040ef2c     LIBCMT:timeset.obj
 0003:00000f30       __dstbias                  0040ef30     LIBCMT:timeset.obj
 0003:00000fb8       __tzname                   0040efb8     LIBCMT:timeset.obj
 0003:00000fe0       __lpdays                   0040efe0     LIBCMT:days.obj
 0003:00001014       __days                     0040f014     LIBCMT:days.obj
 0003:00001140       __cflush                   0040f140     LIBCMT:_file.obj
 0003:00001144       __aenvptr                  0040f144     LIBCMT:crt0.obj
 0003:00001148       __wenvptr                  0040f148     LIBCMT:crt0.obj
 0003:0000114c       ___error_mode              0040f14c     LIBCMT:crt0.obj
 0003:00001474       __maxwait                  0040f474     LIBCMT:crtheap.obj
 0003:00001478       __umaskval                 0040f478     LIBCMT:crt0dat.obj
 0003:0000147c       __osplatform               0040f47c     LIBCMT:crt0dat.obj
 0003:00001480       __osver                    0040f480     LIBCMT:crt0dat.obj
 0003:00001484       __winver                   0040f484     LIBCMT:crt0dat.obj
 0003:00001488       __winmajor                 0040f488     LIBCMT:crt0dat.obj
 0003:0000148c       __winminor                 0040f48c     LIBCMT:crt0dat.obj
 0003:00001490       ___argc                    0040f490     LIBCMT:crt0dat.obj
 0003:00001494       ___argv                    0040f494     LIBCMT:crt0dat.obj
 0003:00001498       ___wargv                   0040f498     LIBCMT:crt0dat.obj
 0003:0000149c       __environ                  0040f49c     LIBCMT:crt0dat.obj
 0003:000014a0       ___initenv                 0040f4a0     LIBCMT:crt0dat.obj
 0003:000014a4       __wenviron                 0040f4a4     LIBCMT:crt0dat.obj
 0003:000014a8       ___winitenv                0040f4a8     LIBCMT:crt0dat.obj
 0003:000014ac       __pgmptr                   0040f4ac     LIBCMT:crt0dat.obj
 0003:000014b0       __wpgmptr                  0040f4b0     LIBCMT:crt0dat.obj
 0003:000014b4       __exitflag                 0040f4b4     LIBCMT:crt0dat.obj
 0003:000014b8       __C_Termination_Done       0040f4b8     LIBCMT:crt0dat.obj
 0003:000014bc       __C_Exit_Done              0040f4bc     LIBCMT:crt0dat.obj
 0003:00001610       ___pInvalidArgHandler      0040f610     LIBCMT:invarg.obj
 0003:00001614       __stdbuf                   0040f614     LIBCMT:_sftbuf.obj
 0003:00001a44       _gpFlsAlloc                0040fa44     LIBCMT:tidtable.obj
 0003:00001a48       _gpFlsGetValue             0040fa48     LIBCMT:tidtable.obj
 0003:00001a4c       _gpFlsSetValue             0040fa4c     LIBCMT:tidtable.obj
 0003:00001a50       _gpFlsFree                 0040fa50     LIBCMT:tidtable.obj
 0003:00001a54       __crtheap                  0040fa54     LIBCMT:heapinit.obj
 0003:00001a5c       ___sbh_pHeaderDefer        0040fa5c     LIBCMT:sbheap.obj
 0003:00001a60       ?__pInconsistency@@3P6AXXZA 0040fa60     LIBCMT:hooks.obj
 0003:00001a84       ___pPurecall               0040fa84     LIBCMT:inithelp.obj
 0003:00001a88       ?_pnhHeap@@3P6AHI@ZA       0040fa88     LIBCMT:handler.obj
 0003:00001a8c       __commode                  0040fa8c     LIBCMT:ncommode.obj
 0003:00001a94       ___mbulinfo                0040fa94     LIBCMT:mbctype.obj
 0003:00001aa0       ___mbcodepage              0040faa0     LIBCMT:mbctype.obj
 0003:00001aa4       ___ismbcodepage            0040faa4     LIBCMT:mbctype.obj
 0003:00001aa8       ___mblcid                  0040faa8     LIBCMT:mbctype.obj
 0003:00001aac       ___locale_changed          0040faac     LIBCMT:setlocal.obj
 0003:00001ab0       ___lc_handle               0040fab0     LIBCMT:nlsdata2.obj
 0003:00001ac8       ___lc_codepage             0040fac8     LIBCMT:nlsdata2.obj
 0003:00001acc       ___lc_collate_cp           0040facc     LIBCMT:nlsdata2.obj
 0003:00001ae8       __newmode                  0040fae8     LIBCMT:_newmode.obj
 0003:00001af4       ___lconv_static_null       0040faf4     LIBCMT:lconv.obj
 0003:00001af8       __fmode                    0040faf8     LIBCMT:txtmode.obj
 0003:00001bb8       ___use_sse2_mathfcns       0040fbb8     <common>
 0003:00001bbc       ___sse2_available          0040fbbc     <common>
 0003:00001bc0       ___sbh_cntHeaderList       0040fbc0     <common>
 0003:00001bc4       ___sbh_pHeaderList         0040fbc4     <common>
 0003:00001bc8       ___sbh_threshold           0040fbc8     <common>
 0003:00001bcc       ___sbh_pHeaderScan         0040fbcc     <common>
 0003:00001bd0       ___sbh_sizeHeaderList      0040fbd0     <common>
 0003:00001bd4       ___sbh_indGroupDefer       0040fbd4     <common>
 0003:00001bd8       __debugger_hook_dummy      0040fbd8     <common>
 0003:00001bdc       ___active_heap             0040fbdc     <common>
 0003:00001be0       __pDestructExceptionObject 0040fbe0     <common>
 0003:00001be4       ___env_initialized         0040fbe4     <common>
 0003:00001be8       ___onexitend               0040fbe8     <common>
 0003:00001bec       ___onexitbegin             0040fbec     <common>
 0003:00001bf0       ___mbctype_initialized     0040fbf0     <common>
 0003:00001bf4       __FPinit                   0040fbf4     <common>
 0003:00001bf8       ___dyn_tls_init_callback   0040fbf8     <common>
 0003:00001bfc       __nhandle                  0040fbfc     <common>
 0003:00001c00       ___pioinfo                 0040fc00     <common>
 0003:00001d00       __acmdln                   0040fd00     <common>
 0003:00001d04       ___piob                    0040fd04     <common>
 0003:00001d20       __bufin                    0040fd20     <common>
 0003:00002d20       __nstream                  00410d20     <common>

 entry point at        0001:00000a26

 Static symbols

 0001:00000000       _hexdump                   00401000 f    CIL library: CIL module
 0001:0000080b       _fast_error_exit           0040180b f   LIBCMT:crt0.obj
 0001:0000082f       _check_managed_app         0040182f f   LIBCMT:crt0.obj
 0001:00000870       ___tmainCRTStartup         00401870 f   LIBCMT:crt0.obj
 0001:00000fe5       __initterm                 00401fe5 f   LIBCMT:crt0dat.obj
 0001:00001122       _doexit                    00402122 f   LIBCMT:crt0dat.obj
 0001:00001334       _flsall                    00402334 f   LIBCMT:fflush.obj
 0001:00001f08       __unwind_handler4          00402f08 f   LIBCMT:exsup4.obj
 0001:00002112       _write_char                00403112 f   LIBCMT:output.obj
 0001:00002145       _write_multi_char          00403145 f   LIBCMT:output.obj
 0001:00002169       _write_string              00403169 f   LIBCMT:output.obj
 0001:00003132       _parse_cmdline             00404132 f   LIBCMT:stdargv.obj
 0001:00003500       __use_encode_pointer       00404500 f   LIBCMT:tidtable.obj
 0001:00003c17       ___crtInitCritSecNoSpinCount@8 00404c17 f   LIBCMT:initcrit.obj
 0001:00004c36       __onexit_nolock            00405c36 f   LIBCMT:onexit.obj
 0001:00004f2e       _siglookup                 00405f2e f   LIBCMT:winsig.obj
 0001:0000606a       __tsopen_nolock            0040706a f   LIBCMT:open.obj
 0001:00006c7c       __unwind_handler           00407c7c f   LIBCMT:exsup.obj
 0001:00006df1       ?CPtoLCID@@YAHH@Z          00407df1 f   LIBCMT:mbctype.obj
 0001:00006e20       ?setSBCS@@YAXPAUthreadmbcinfostruct@@@Z 00407e20 f   LIBCMT:mbctype.obj
 0001:00006e75       ?setSBUpLow@@YAXPAUthreadmbcinfostruct@@@Z 00407e75 f   LIBCMT:mbctype.obj
 0001:000070a3       ?getSystemCP@@YAHH@Z       004080a3 f   LIBCMT:mbctype.obj
 0001:00007700       __updatetlocinfoEx_nolock  00408700 f   LIBCMT:setlocal.obj
 0001:00008371       ?x_ismbbtype_l@@YAHPAUlocaleinfo_struct@@IHH@Z 00409371 f   LIBCMT:ismbbyte.obj
 0001:00009084       _fastzero_I                0040a084 f   LIBCMT:p4_memset.obj
 0001:00009494       ?__crtLCMapStringA_stat@@YAHPAUlocaleinfo_struct@@KKPBDHPADHHH@Z 0040a494 f   LIBCMT:a_map.obj
 0001:00009a3f       ?__crtGetStringTypeA_stat@@YAHPAUlocaleinfo_struct@@KPBDHPAGHHH@Z 0040aa3f f   LIBCMT:a_str.obj
 0001:00009f20       ?strtoxl@@YAKPAUlocaleinfo_struct@@PBDPAPBDHH@Z 0040af20 f   LIBCMT:strtol.obj
 0001:0000a174       _fastcopy_I                0040b174 f   LIBCMT:p4_memcpy.obj
 0001:0000a418       _has_osfxsr_set            0040b418 f   LIBCMT:cpu_disp.obj
